:020000040000FA
:0400000028EF00F0F5
:02000800B3D073
:0800180047D0086A076EFF0ED5
:100020000726082200D0D8A01200030E066EE60EA6
:1000300002D8F5D7066AFE0F056E000000D000D08A
:10004000E86A065AD8A01200050600D000D0F5D7FD
:10005000F86AAB6AAC6A7B6A7A6A7E6A7F6AC26A4D
:10006000A66AA68EF19E7B6A7A6A7E6A0F0EC16EC0
:10007000926A936A946A210E926E9368800E946ECF
:10008000926A806AD56AD58CD586F28AF194D66A4E
:10009000D76A7D88F286F180F28EF28CD08ED59E62
:1000A000F290640EBADFDFD0F29ED8CFF1F5E8CF40
:1000B000F2F5E0CFF3F5E9CFF4F5EACFF5F5E1CFCE
:1000C000F6F5E2CFF7F5D9CFF8F5DACFF9F5F6CFB7
:1000D000FAF5F7CFFBF5F5CFFCF5F3CFFDF5F4CF4F
:1000E000FEF5A6CFFFF5F28E0001F2A41FD0F29428
:1000F000D59E105203E08086100601D080961152E2
:1001000003E08082110601D08092125203E08084C5
:10011000120601D08094172A1750166207D00DC01E
:1001200010F00EC011F00FC012F0176AD58EF29EBB
:10013000F1C5D8FFF2C5E8FFF3C5E0FFF4C5E9FF5C
:10014000F5C5EAFFF6C5E1FFF7C5E2FFF8C5D9FF3F
:10015000F9C5DAFFFAC5F6FFFBC5F7FFFCC5F5FFE9
:10016000FDC5F3FFFEC5F4FFFFC5A6FFF28E10002C
:10017000D8CF0BF00C6EE0CF00F0E9CF01F0EACF62
:1001800002F00001F2A010D0D59E8150F29081B80B
:100190000BD081A8FED70A0E40DF1D2A1D2C02D0ED
:1001A0000DD002D01D6AFF0001C0E9FF02C0EAFFC6
:1001B00000C0E0FF0C500BC0D8FF10008150F2903F
:1001C000F28E00D082BE09D082AEFED70A0E25DFA5
:1001D0001C2A070E1C6201D01C6A1C5207E1929671
:1001E000898692928982929489843AD01C2C07D075
:1001F00092968986929289929294898431D0020E45
:100200001C6207D0929689869292899292948994E0
:1002100027D0030E1C6207D092968986929289821B
:10022000929489941DD0040E1C6207D092968996F0
:10023000929289829294899413D0050E1C6207D001
:1002400092968996929289829294898409D0060E18
:100250001C6206D092968996929289929294898491
:100260000A0EDBDEAFD71C6A1D6A1668640E186EB4
:100270001A6AD58E9FD01A50060DF3CF19F0030ECF
:10028000046ED60E036E19500324F66E000E042081
:10029000F76E0800F5CF0DF0030E046ED60E036E58
:1002A00019500324096E000E04200A6E010E092461
:1002B000F66E000E0A20F76E0800F5CF13F0030E5D
:1002C000046ED60E036E19500324096E000E04202E
:1002D0000A6E020E0924F66E000E0A20F76E080060
:1002E000F5CF0EF0030E046ED60E036E19500324E4
:1002F000096E000E04200A6E030E0924F66E000E2D
:100300000A20F76E0800F5CF14F0030E046ED60E27
:10031000036E19500324096E000E04200A6E040EA9
:100320000924F66E000E0A20F76E0800F5CF0FF0D4
:10033000030E046ED60E036E19500324096E000ED0
:1003400004200A6E050E0924F66E000E0A20F76ED0
:100350000800F5CF15F012001352D8B40CD0132CAE
:1003600004D00D4801D00D2A06D0020E136203D02E
:100370000D52D8A40D061452D8B40CD0142C04D0AD
:100380000E4801D00E2A06D0020E146203D00E527F
:10039000D8A40E061552D8B40CD0152C04D00F4892
:1003A00001D00F2A06D0020E156203D00F52D8A436
:1003B0000F06120081501A6A060E1A6009D05BDF20
:1003C0001B6A0A0E2ADEC8DF1B2AFBE11A2AF4E1A7
:1003D0000A0E23DEEFD7FF0000010000FF02FF003E
:1003E00000000000FF0000010000FF02FF0000010C
:0C03F0000000FF00FF000000FF02FFD72C
:020000040030CA
:0300010006190ECF
:020005008180F8
:060008000FC00FE00F40E5
:00000001FF
